:020000040800F2
:10000000E842002001010008992E0008891C000820
:10001000152D0008F9010008A534000800000000B3
:100020000000000000000000000000003730000861
:1000300031020008000000009B2E00082931000852
:100040001B0100081B0100081B0100081B01000820
:100050001B0100081B0100081B0100081B01000810
:100060001B0100081B0100081B0100081B01000800
:100070001B0100081B0100081B0100081B010008F0
:100080001B0100081B0100081B0100081B010008E0
:100090001B0100081B0100081B0100081B010008D0
:1000A0001B0100081B0100081B0100081B010008C0
:1000B0008931000895310008A1310008991C000819
:1000C0008D1C00081B0100081B0100081B01000813
:1000D0001B0100088D3400081B010008993400083A
:1000E0001B0100081B0100081B010008DFF80CD0F1
:1000F00000F03CF800480047FD340008E8420020CA
:100100000648804706480047FEE7FEE7FEE7FEE7B1
:10011000FEE7FEE7FEE7FEE7FEE7FEE787310008C1
:10012000ED00000840EA01039B0703D009E008C97D
:10013000121F08C0042AFAD203E011F8013B00F8AC
:10014000013B521EF9D27047D2B201E000F8012BF8
:10015000491EFBD270470022F6E710B513460A4647
:1001600004461946FFF7F0FF204610BD064C074D28
:1001700006E0E06840F0010394E807009847103477
:10018000AC42F6D3FFF7B6FFD8360008F8360008C1
:1001900010B50446142003F037FAA02104608180D2
:1001A0004FF4007181604021C16049020182022147
:1001B000C18041820149086010BD00002C00002070
:1001C0003EB50C4B1C689CB18318B3F5004F0DD2A3
:1001D0004FF6FF738DE80E00A188E388246802467D
:1001E00041F00101204600F0DFFB014608463EBD1C
:1001F00001203EBD2C000020FEE70000044B01283A
:1002000001D0002200E001220421184600F07FB94D
:10021000000C0140054B4FF40051012801D0002291
:1002200000E00122184600F072B90000000C014005
:10023000704772B6FEE710B590F82110002202292F
:1002400005D00421816380F82020012010BD0168C1
:100250000B6823F00E030B6001680B6823F00103A9
:100260000B6090F84030C46B012101FA03F3636026
:1002700080F8211080F82020104610BD10B590F8AD
:1002800021100024022903D00421816301243DE0D0
:1002900001680A6822F00E020A6001680A6822F00A
:1002A00001020A601A4A0168914201D1012121E04C
:1002B000174A1432914201D110211BE0144A28320E
:1002C000914201D1891515E0114A3C32914201D188
:1002D00089140FE00E4A5032914202D14FF480311E
:1002E00008E00B4A6432914202D14FF4801101E0E0
:1002F0004FF08071064A083A5160012180F82110C0
:10030000002180F82010416B01B18847204610BDC4
:100310000800024090F82100704700002DE9F84FD6
:10032000DFF8B0910024A9F1040B23460F2709F14F
:10033000040AABF1040EC6E00125A5402A40AA42FA
:1003400076D1DFF894C14E68A6EB0C0866452BD039
:100350000DDC032E34D005DC36B3012E19D0022E6D
:100360002FD11BE0112E16D0122E2AD119E0B8F58C
:10037000881F19D006DCB8F5803F15D0B8F5801F6E
:100380001FD111E0B8F5001F0ED0B8F5041F18D129
:100390000AE0CB6815E0CB681B1D12E0CB68083380
:1003A0000FE0CB680C330CE08B682BB1012B4FF0C6
:1003B000080303D0456104E0042302E0056100E086
:1003C0000023FF2A01D8064601E000F104064FEAA7
:1003D000840501D9A5F12005D6F8008007FA05FCAF
:1003E00028EA0C0803FA05F548EA0508C6F8008073
:1003F0004D68ED0066D5394DAE6946F00106AE6137
:10040000AD6924F0030605F001050095344D06EBB7
:10041000050CDCF80850A607360F07FA06F825EA9F
:100420000805DFF8C080404503D14FF0000817E011
:1004300048E0DFF8B480404502D14FF001080FE0FA
:10044000DFF8A880404502D14FF0020808E0DFF84D
:10045000A080404502D14FF0030801E04FF00408AE
:1004600008FA06F848EA0508CCF808804D68D9F87B
:100470000060ED02002D4D4601DA164300E0964380
:100480002E604D68DAF80060AD02002D554601DAA5
:10049000164300E096432E604D68DBF80060AD0324
:1004A000002D5D4601DA164300E096432E604D684C
:1004B000DEF80060ED03002D754601DA164300E01A
:1004C00096432E60641C0A6832FA04F57FF434AF58
:1004D000BDE8F88F08040140000011100010024030
:1004E0000000014000080140000C014000100140E4
:1004F000001401408068084000D001207047C268A5
:1005000021EA02030A4043EA0241016170470AB14D
:10051000016170470904FBE70148806870470000EB
:100520000C000020704770472DE9F0410168044637
:100530004A694E6890F83E000025D743FA050BD46F
:10054000F243D20508D46FF4807201254A61216814
:100550000A6842F400420A60B90508D4F143C905AB
:1005600005D422686FF4007145F0020551617905E8
:1005700025D4F143C90522D4638D94F83D10226B34
:10058000202808D13BB9212910D029290ED02829AB
:1005900001D1212A0AD022686FF48061516145F0AF
:1005A0000405102806D0402804D008E0204602F0B8
:1005B0000DF804E02068016841F40071016038051D
:1005C00008D4F043C00505D421686FF4006045F0FD
:1005D00008054861002D07D0206C28432064204680
:1005E000BDE8F04101F0C4BBBDE8F0812DE9F04762
:1005F000026800215368C66A90F83E4090F83D506A
:10060000102C12D0402C10D0046C002C7DD05469DA
:10061000E443A6077AD4DE43B60577D4036C03B16E
:100620009169BDE8F04701F0ADBF976951694FF49A
:100630002A0CC9435FEAC1784FF02A4904D06645C5
:100640002AD04E4528D010E0DE43B6050DD4C16A4D
:10065000614501D1012103E0C16A494501D1082169
:10066000C162BDE8F04701F075BE0E0716D4DE4347
:10067000B60513D4416CC9B21161416B09B1896AE5
:1006800029B9816B002907D0896A002904D0006844
:10069000416841F400614160BDE8F0878E0706D4EF
:1006A000DE43B60503D4BDE8F04701F0A7BDFE4325
:1006B000526876074FEA02521DD4002AECDB0A0684
:1006C00008D4DA43520505D4490705D5BDE8F047FB
:1006D00001F039BD4907DFD4D9438905DCD4212D88
:1006E00005D0402CD8D1BDE8F04701F079BEBDE877
:1006F000F04701F0E7BC002ACEDB4A060BD4DA4310
:10070000520508D4490708D501E00DE00EE0BDE828
:10071000F04701F05DBC4907BED4D9438905BBD47D
:10072000BDE8F04701F0E7BB916970E7E10606D448
:10073000D943890503D4BDE8F04701F08FBF2821D4
:10074000212D27D0292D25D0650655D4DD436D05F3
:1007500052D4640752D590F83D30448D002C9BD084
:100760001269446A2270426A521C4262428D521ED1
:100770004285428D002A8FD12A2B8DD10268536881
:1007800023F4806353602222026380F83D1000F05E
:100790007DFA81E7250623D4DD436D0520D4640767
:1007A00020D590F83D30448D002CF2D0446A247856
:1007B0001461426A521C4262428D521E4285428D31
:1007C000002AE6D1292BE4D10268536823F4806320
:1007D00053602122026380F83D1000F058FA5BE775
:1007E0006107D6D4D9438905D3D4418D0029D0D00F
:1007F000416A097811610AE06107CAD4D9438905C1
:10080000C7D4418D0029C4D01169426A1170416A70
:10081000491C4162418D491E41853DE770470000FA
:1008200070B5040025D094F83D00002520B984F867
:100830003C50204600F0ECF9242084F83D0020686C
:10084000016821F0010101602068016841F4004164
:1008500001602068016821F40041016000F092FB12
:100860004A4A6168914201D8494900E049498842B1
:1008700001D2012070BD48492368B0FBF1F15E68E8
:1008800026F03F060E435E606368934206D94FF43C
:10089000967359434FF47A73B1FBF3F12368491C03
:1008A0001E6A26F03F0631431962616891420AD8F8
:1008B0004900401EB0FBF1F0401CC0F30B000428BF
:1008C0001ED204201CE0A368F3B301EBC10202EBCB
:1008D0000116421EB2FBF6F2521C42F4804212058F
:1008E00049D093B301EBC10202EB0111401EB0FBF2
:1008F000F1F0401CC0F30B0040F4804040F4004095
:100900002168CA694CF6FF739A431043C861D4E961
:10091000071001432068026822F0C0021143016001
:10092000D4E9030101432068826848F2FF339A4307
:1009300011438160D4E9050108432168CA6822F0A7
:10094000FF021043C86001E00EE016E02068016875
:1009500041F0010101602564202084F83D002563F9
:1009600084F83E50002070BD01EB4106421EB2FBF0
:10097000F6F2521CB3E70120C2E701EB4101401E31
:10098000B0FBF1F0401CC0F30B00B7E7A0860100FC
:1009900080841E0000093D0040420F0070477047F0
:1009A00070477047704700002DE9FF4F83B0002566
:1009B000DDE910799A4693460446DDF848800095B3
:1009C000FFF7AAFD064694F83D0020287DD11923A3
:1009D00001228B492046009601F0F0FE0028F5D157
:1009E00094F83C00012870D0012084F83C00206875
:1009F0000168C90703D1016841F001010160206865
:100A0000016821F400610160222084F83D0040204B
:100A100084F83E0025646762A4F82A90608D2085E2
:100A20007848E062CDE9008653465A46204604994C
:100A300001F02AFD00287DD1208DDFF8CC91202700
:100A400068B1012814D00228206801681ED041F442
:100A5000806101602068416980690090C5E020687C
:100A6000416981690091016841F400710160BCE055
:100A70002068016821F48061016072B620684169D4
:100A800081690091016841F400710AE041F400615C
:100A9000016072B62068416981690091016821F4A2
:100AA0008061016062B6A0E003286AD801280DD0F9
:100AB000022843464FF000024946204600960CD0DB
:100AC00001F07CFE002862D10CE097E032464146FE
:100AD000204601F019FF68BB7AE001F06FFE48BBC9
:100AE00072B637E02068016821F48061016072B657
:100AF00020680069616A0870606A00F10100606244
:100B0000208DA0F101002085608DA0F1010060859D
:100B10003E4846F2A8110068B0FBF1F0C0EBC000FF
:100B200000EB80000090401E009008D020684069D3
:100B3000C04300E02BE040070CD50098F3E744F8F1
:100B4000305F6773A573206940F02000206162B6B2
:100B500025731CE02068016841F400710160206881
:100B60000069616A0870606A401C6062218D491EDC
:100B70002185618D491E618562B621680969017010
:100B80002AE032464146204601F0BEFE18B101205F
:100B900007B0BDE8F08F20680069616A0870606A7C
:100BA00000F101006062208DA0F1010081B2218579
:100BB000608DA0F101006085206842696FEA020241
:100BC000520712D4032903D1016821F48061016026
:100BD00020680069616A0870606A401C6062208D4C
:100BE000401E2085608D401E6085208D00287FF48A
:100BF0005BAF3C346770A5702570C9E70220C7E77A
:100C0000020010000000FFFF040001001800002097
:100C100010B586B000210091019102910391006806
:100C2000174988422AD1174CA06940F00800A061FA
:100C3000A069694600F008000490C02000901220CE
:100C40000190032003901048FFF768FBE06940F42F
:100C50000010E061E069002200F4001004901146E9
:100C60001F2000F0A7F81F2000F096F80022114680
:100C7000202000F09FF8202000F08EF806B010BD74
:100C80000054004000100240000C014070477047C3
:100C90000248816802781144816070470C0000208E
:100CA000074810B5016841F010010160032000F011
:100CB000A1F80F2000F006F800F050F8002010BD59
:100CC0000020024030B505461F4887B0C16941F099
:100CD0000401C161C06906A900F00400009001A8E8
:100CE00000F030F90498B0B100F04CF94000174919
:100CF000174AB0FBF1F11748491E0260416040F20B
:100D0000E7320021C0E903218160816100F04AFBE4
:100D1000040003D015E000F035F9E8E70D4800F0D5
:100D200095FB04000DD11E2000F036F8102D07D2DF
:100D3000002229461E2000F03DF80748056000E02B
:100D4000012407B0204630BD0010024040420F0091
:100D50000008004014020020100000200C4808B5D4
:100D6000816941F001018161816901F00101009116
:100D7000C16941F08051C161C06900F080500090AC
:100D80000448416821F0E06141F00071416008BD14
:100D9000001002400000014000280ADB00F01F02A2
:100DA0000121914040094FF0E02202EB8000C0F8A1
:100DB00000117047F0B40E4B1B680C46C3F30223BE
:100DC000C3F10705042D00D90425191D072901D2F7
:100DD000002300E0DB1E012606FA05F1491E214032
:100DE00099409E40761E16403143F0BC02F05CBB39
:100DF0000CED00E0064900F0070208684FF6FF031B
:100E0000184040EA0220034A10430860704700007F
:100E10000CED00E00000FA052DE9F0470F46050053
:100E200061D0434E306800F00700B84209D2306804
:100E300020F0070038433060306800F00700B84207
:100E400051D128683B4C810712D5400703D5606813
:100E500040F4E06060602878000703D5606840F4E3
:100E6000605060606068A96820F0F000084360602E
:100E70002878C00728D06868012810D02168022887
:100E800010D0890700292EDA616821F0030101439F
:100E90006160FFF741FB804641F288390DE021682F
:100EA0008903EFE78901EDE7FFF736FBA0EB0801C7
:100EB000494502D90320BDE8F0876068696800F001
:100EC0000C00B0EB810FEFD1306800F00700B842A2
:100ED0000BD9306820F0070038433060306800F0EC
:100EE0000700B84201D00120E5E72878400705D582
:100EF0006068E96820F4E0600843606028780007D3
:100F000006D56068296920F4605040EAC10060603D
:100F100000F058F86168084AC1F30311515CC840F9
:100F20000649086006480068FFF7CCFE0020C2E7CB
:100F30000020024000100240BE36000818000020C9
:100F4000100000200F2202600C4A536803F00303D4
:100F50004360536803F0F0038360536803F4E06375
:100F6000C36052684FF4E06303EAD20202610448AE
:100F7000006800F0070008607047000000100240A1
:100F8000002002400448054900684968044AC1F34A
:100F90000221515CC8407047180000200010024038
:100FA000CE3600080448054900684968044AC1F380
:100FB000C221515CC8407047180000200010024058
:100FC000CE3600080E4A51680E4801F00C03042B7F
:100FD00011D0082B0FD10C48C1F38343C903C05C67
:100FE0000AD55168084AC1F34041921E515C054A36
:100FF0005043B0FBF1F0704704494843704700008C
:101000000010024000127A00AE36000800093D00D0
:101010002DE9F84F040070D02078C24DC00749D0A8
:101020006868C0F38100012807D06868C0F38100B8
:10103000022809D16868C00306D52868800339D51D
:1010400060680028E7D035E06068B0F5803F0BD0DD
:1010500010B1B0F5A02F11D0286820F4803028609E
:10106000286820F4802002E0286840F4803028605E
:10107000606890B1FFF750FA06460AE0286840F42D
:1010800080202860F0E700BFFFF746FA801B642845
:1010900074D828688003F7D50CE0FFF73DFA0646C0
:1010A00005E000BFFFF738FA801B6428F0D82868F5
:1010B0008003F7D420789C4E80074FF001094FF051
:1010C000000839D5686810F00C0F07D06868C0F3C5
:1010D0008100022809D16868C00306D42868800707
:1010E00014D52069012808D110E02069B0B1C6F8F4
:1010F0000090FFF711FA074605E00EE1FFF70CFA42
:10110000C01B0228C4D828688007F7D52868616901
:1011100020F0F80040EAC10028600DE0C6F8008029
:10112000FFF7FAF9074604E0FFF7F6F9C01B0228BB
:10113000AED828688007F7D4207800072ED57B48E2
:10114000A169E1B1C0F80090FFF7E6F9074604E0B5
:10115000FFF7E2F9C01B022810D8686A8007F7D5AC
:1011600073484FF4FA510068B0FBF1F0009000BFF3
:101170000098411E00910028F9D10FE082E0C0F8EC
:101180000080FFF7C9F9074605E000BFFFF7C4F983
:10119000C01B022876D8686A8007F7D420784007F9
:1011A00061D5E8690027C00008D4E86940F08050A4
:1011B000E861E869012700F0805000905D4801680F
:1011C000C90513D40168834641F480710160FFF7BB
:1011D000A3F9824606E000BFFFF79EF9A0EB0A00E4
:1011E00064284FD8DBF80000C005F5D5E068012879
:1011F0000AD008B1052813D0286A20F0010028621F
:10120000286A20F0040002E0286A40F00100286209
:10121000E06841F2883B98B1FFF77EF982460BE027
:10122000286A40F004002862EEE700BFFFF774F977
:10123000A0EB0A0159455CD8286A8007F6D50CE076
:10124000FFF76AF9824605E0FFF766F9A0EB0A01AD
:1012500059454ED8286A8007F6D4012F03D1E86992
:1012600020F08050E861E06990B36968C1F38101C2
:10127000022945D00228C6F8608004D0FFF74CF957
:10128000044639E035E0FFF747F9074605E000BFBF
:10129000FFF742F9C01B02282BD828688001F7D439
:1012A000206AB0F5803F05D16868A16820F400305D
:1012B00008436860D4E908010843696821F474119F
:1012C00008436860C6F86090FFF726F9044606E018
:1012D00025E000BFFFF720F9001B022809D8286885
:1012E0008001F7D51BE000BFFFF716F9001B0228AD
:1012F00002D90320BDE8F88F28688001F4D40EE0FD
:101300000128F7D06868226A00F48031914204D144
:10131000616A00F47010884201D00120EAE70020E1
:10132000E8E7000000100240000042428004424210
:1013300018000020007000407047704770B590F8AA
:101340003C20012A25D0012480F83C40022280F86C
:101350003D2003685A689D6822F070060A6832438F
:101360005A600D4B02689A4208D0B2F1804F05D006
:101370000A4B9A4202D00A4B9A4204D1496825F09E
:101380008003194391603C3044700021017008468D
:1013900070BD022070BD0000002C01400004004020
:1013A0000008004010B5040003D094F83D0010B1CF
:1013B00007E0012010BD002084F83C00204600F02A
:1013C00015F8022084F83D00211D206801F0EEFE92
:1013D00001203D3460726070A070E0702071607117
:1013E000A071E07120722070002010BD08B5016866
:1013F0001448B1F1804F14D0134A914220D1C169F1
:1014000041F00201C161C069002200F002000090B9
:1014100011461D20FFF7CEFC1D20BDE80840FFF758
:10142000BBBCC16941F00101C161C069002200F08B
:101430000100009011461C20FFF7BCFC1C20ECE7CB
:1014400008BD0000001002400004004090F83D106C
:10145000012901D001207047022180F83D10016868
:10146000CA6842F00102CA6000680B49884208D08D
:10147000B0F1804F05D00949884202D0084988421E
:1014800004D1816801F00701062903D0016841F009
:101490000101016000207047002C01400004004061
:1014A0000008004070B5044690F83C000025012873
:1014B00017D0012684F83C60022084F83D002068A3
:1014C000826822F0770222F47F4282600868502806
:1014D00037D00DDC20284ED005DC88B3102811D180
:1014E00049E0022070BD302845D040280AD13AE0BA
:1014F00060282ED070280CD0B0F5805F03D0B0F5F6
:10150000005F11D001253C34667000202070284611
:1015100070BD4A68083120680AC901F083FE20685E
:10152000816841F0770109E04A68083120680AC9FA
:1015300001F078FE2068816841F480418160E2E733
:1015400019E0CA684968206801F07EFE50212068D1
:1015500006E0CA684968206801F087FE60212068BB
:1015600001F06AFECFE7CA684968206801F06CFEA6
:1015700040212068F4E7226801461046F0E77047F2
:101580002DE9F04104460068C66805694FF0000780
:10159000A90713D5B10711D5F91E016101202077E4
:1015A000206880698007204602D0FFF7E8FF04E04A
:1015B00000F07EF8204600F07CF82777680716D503
:1015C000700714D521686FF00400086102202077AD
:1015D0002068806910F4407F204602D0FFF7CFFFDB
:1015E00004E000F065F8204600F063F8277728074C
:1015F00015D5300713D521686FF008000861042065
:1016000020772068C0698007204602D0FFF7B7FF27
:1016100004E000F04DF8204600F04BF82777E8068C
:1016200016D5F00614D521686FF010000861082067
:1016300020772068C06910F4407F204602D0FFF771
:101640009EFF04E000F034F8204600F032F82777DF
:10165000E80708D0F00706D021686FF001000861A4
:10166000204600F027F8280608D5300606D5216860
:101670006FF0800008612046FFF75EFE680608D51F
:10168000700606D521686FF040000861204600F022
:101690001FF8A8060AD5B00608D521686FF020000B
:1016A00008612046BDE8F041FFF747BEBDE8F08184
:1016B0007047704700680549884201D1FFF7E8BAD2
:1016C000B0F1804F01D101F0D5BF70470008004054
:1016D000704718B5034690F84200202801D0022038
:1016E00018BD61B15AB10120186300205863184633
:1016F00001F0B0FE0028F3D1196B012901D00120BF
:1017000018BD19680A684968009119680C3151E8D8
:10171000002F42F0100241E80024002CF5D118BD42
:101720000F4A136819E05A68824215D159B1D86836
:1017300008445969884200D3401AD8601969884220
:1017400001D101201877998AD868091A8AB2996854
:1017500001445868FFF7BDBF1B6C002BE3D17047F5
:101760001C0000207047000070B5044620680C3053
:1017700050E8001F21F4907140E80012002AF5D1D2
:101780002068143050E8001F21F0010140E80012E9
:10179000002AF5D1206B01280AD1206800F10C0045
:1017A00050E8001F21F0100140E80012002AF4D197
:1017B000206840694FF0200241064FF0000015D527
:1017C0002168143151E8003F23F0400341E800351F
:1017D000002DF5D1E16B49B109484863E06BFEF794
:1017E0004DFD50B1E06B416B884706E0E08584F821
:1017F000422020632046FFF7B5FF002070BD0000A7
:101800009F32000838B5416C002924D012490C6879
:101810001FE0616881421BD1002184F83910A16268
:10182000006801684068009060680068016841686D
:101830000091C16821F02001C1606068FFF794FF4A
:10184000A08A82B2D4E90101BDE83840FFF741BF68
:10185000246C002CDDD138BD1C000020F8B50168D7
:1018600004460868CA684B6910F00F0F4FF0000576
:101870005AD003F0010602F49077374365D0C107D0
:1018800005D0D10503D5616C41F0010161644107C8
:1018900005D5D90703D0616C41F00201616481076D
:1018A00005D5D90703D0616C41F0040161640107DB
:1018B00007D502F02001314303D0616C41F00801EB
:1018C0006164616C00293BD0800604D5900602D586
:1018D000204601F016FD20684069616CC0F380105D
:1018E00001F00801014320462BD001F0E3FC206801
:1018F0004069400621D52068143050E8001F21F0CF
:10190000400140E80012002AF5D1E06BA8B16E4911
:101910004163E06BFEF7B2FC002811D0E06B416B35
:1019200001B0BDE8F040084783060ED593060CD5FC
:101930002046BDE8F84001F0E4BC2046FFF762FF16
:10194000F8BDFFF75FFF6564F8BD266B2023012E0D
:101950007CD1C6067AD5D60678D508684868009046
:1019600048694FF00206400640D5E16B08684068C0
:101970000004000CE8D0A28D8242E5D9E085886998
:1019800020282DD020680C3050E8001F21F48071F1
:1019900040E80012002AF5D12168143151E8000F07
:1019A00020F0010041E80002002AF5D1206814303F
:1019B00050E8001F21F0400140E80012002AF5D154
:1019C00084F84230256320680C3050E8001F21F075
:1019D000100140E80012002AF5D1E06BFEF72BFC65
:1019E0006663A08DE18D401A81B22AE0A08DE18D61
:1019F000401A81B2E08D0028A6D00029A4D0226828
:101A00000C3252E8000F20F4907042E80007002FDB
:101A1000F5D12068143050E8002F22F0010240E890
:101A20000027002FF5D184F84230256320680C3060
:101A300050E8002F22F0100240E80023002BF5D1DF
:101A400066632046FFF76CFEF8BDFFE705062CD560
:101A500015062AD594F841002128F5D1A068B0F5E3
:101A6000805F01D12069B0B1206A411C21622168E8
:101A700000784860E08C401E0004000CE084E3D154
:101A80002068C16821F08001C1602068C16841F010
:101A90004001C160D8E7206A0088C0F308004860B0
:101AA000206A00F102002062E4E74006CCD550062F
:101AB000CAD5CA68204622F04002CA6084F8413084
:101AC00000F0D2F8C0E700008F32000870B50400C3
:101AD00004D094F84100002510B106E0012070BD4B
:101AE00084F84050204600F023F8242084F8410078
:101AF0002068C16821F40051C160204601F064FCF7
:101B00002068016921F4904101612068416921F058
:101B10002A0141612068C16841F40051C1606564D7
:101B2000202084F8410084F842006563002070BDE5
:101B300070B586B000240094019402940394036865
:101B40002E482D4E022103220515B34226D183696A
:101B500043F480438361836903F48043049383697E
:101B600043F0040383618069254E00F00400049073
:101B70000802CDE90001039269463046FEF7CEFB2C
:101B8000CDE90054694630460294FEF7C7FB0022B7
:101B900011462520FFF70EF9252028E0194EB34203
:101BA00027D1C36943F48023C361C36903F480234D
:101BB0000493836943F0080383618069CDE9005190
:101BC00000F00800CDE903200F4D69462846FEF7D6
:101BD000A5FBE814CDE90004694628460294FEF707
:101BE0009DFB002211462720FFF7E4F82720FFF78E
:101BF000D3F806B070BD000000380140001002406C
:101C00000008014000480040000C014008490B68F2
:101C10000BE05968814207D10020D860988A82B2CF
:101C2000D3E90101FFF755BD1B6C002BF1D17047C3
:101C30001C00002090F84130202B01D0022070477A
:101C400079B172B101628284C28400214164212190
:101C500080F841100068C16841F08001C160002037
:101C6000704701207047000001460648006805E003
:101C700042688A4201D101F0B1B9006C0028F7D165
:101C8000704700001C000020FEE700000148FEF73E
:101C90004BBC0000A00000200148FEF7A7BC0000DC
:101CA000A000002038B5406A002190F83D202B4B61
:101CB00046F2A8141B68B3FBF4F3C3EBC30303EBB6
:101CC0008303009343B1A3F10103009303681B68EE
:101CD0009B0505D5009BF5E7036C43F020030364E7
:101CE000436B03B19962836B03B1996203681C680B
:101CF00024F480641C604185436B03B15963836B9A
:101D000003B1596303681C6824F001041C6090F857
:101D10003D402023602C0AD0282434EA02020ED051
:101D200080F83D3080F83E10FEF778FD38BD80F831
:101D30003D3080F83E100164FEF7F4FB38BD0268C8
:101D4000136843F0010313600268136843F480636F
:101D50001360016380F83D40E6E7000018000020B2
:101D600000684169C943090601D400210161704737
:101D700070B5044690F83D0094F83E10102901D04B
:101D8000402906D1222804D121680A6822F4006281
:101D90000A60282131EA00024FF000054FF02006CA
:101DA00026D021684968090505D4602803D084F845
:101DB0003D6084F83E50256320684168090537D5A9
:101DC000416821F400614160606B90F821203C493A
:101DD000012A11D04163606BFEF750FA38B32068D6
:101DE000016821F00101016084F83D60606B1CE036
:101DF000256384F83D10DFE7A06B4163A06BFEF71D
:101E00003DFAA0B120684169C943490605D400697B
:101E1000616A0870606A401C60622068016821F095
:101E20000101016084F83D60A06B416B884710E0C0
:101E300094F83D10602910D04169C943490605D482
:101E40000069616A0870606A401C60622046FEF7A3
:101E5000E5FC206CC1071CD115E084F83D602564C9
:101E60004169C943490605D40069616A0870606A1E
:101E7000401C60622068016821F001010160204679
:101E8000FEF750FBE5E7810703D4410701D40007C3
:101E900004D52068416821F4E061416094F83D0078
:101EA000216C49070BD5282809D10648E062256333
:101EB00084F83D6084F83E502046FEF76FFD70BD0B
:101EC000A51C00080000FFFF01684A69D2435205C3
:101ED0000FD46FF480624A61002140F8301F202245
:101EE00042738173026942F00402026101730120AE
:101EF00070470020704710B5C26A438D0168042BFB
:101F000006D0438D032B08D0438D022B1DD012E049
:101F10004A6822F480624A600CE04B6823F48063D4
:101F20004B60042A06D0022A04D001680A6822F411
:101F300080620A6001680969426A1170416A491C3D
:101F40004162418D491E418510BD012A34D0102ABD
:101F500032D0042A34D0022A32D00B6843F4007302
:101F60000B6001680969436A1970416A491C416242
:101F7000438D5B1E438503681B690B70416A491CD6
:101F80004162418D491E418501684B6823F44073CD
:101F90004B60202180F83D1090F83E300021402B0E
:101FA00080F83E1010D0082A02D0202A00D012213A
:101FB0000163FEF7F4FC10BD0B6823F48063CFE7E8
:101FC0000B6843F48063CBE70163FEF7EAFC10BDC6
:101FD00038B590F83D10222910D1C36A418D0329EC
:101FE0000DD901680969426A1170416A491C416250
:101FF000418D491E4185418D032906D038BDC26AF5
:10200000022A02D0012906D029B10068416821F4D2
:102010008061416038BD2A4A46F2A8140021126846
:10202000B2FBF4F202EB8202009202684FF020044D
:10203000009D6D1E009526D01568AD05F8D4156875
:1020400025F4806515600268556825F4E0655560E3
:1020500002681269456A2A70426A521C4262428DC5
:10206000521E428580F83D4090F83E2080F83E1098
:10207000402A21D0082B02D0202B00D0122101634E
:10208000FEF78DFC38BD036C43F0200303645368F6
:1020900023F4E063536002681269436A1A70426A6B
:1020A000521C4262428D521E428580F83D4080F8AB
:1020B0003E10FEF7B3FB38BD0163FEF772FC38BD7E
:1020C0001800002010B5C26A90F83D1021290BD1EC
:1020D000418D51B1416A026809781161416A491C18
:1020E0004162418D491E418510BD20230021082AEF
:1020F00010D0202A0ED012F5803F0BD00268546811
:1021000024F4E06454601122026380F83E1080F8E9
:102110003D3015E00268546824F4E06454600268BD
:10212000146844F400741460016380F83D3090F842
:102130003E2080F83E10402A02D1FEF733FC10BD4D
:10214000FEF72EFC10BD10B590F83D1090F83E3013
:10215000C26A048DB4B1212903D0402B11D12229A8
:102160000FD1418DD9B390F83E10402941D0416A3A
:10217000026809781161416A491C4162418D491E1A
:10218000418510BD2129E8D120230021082A10D043
:10219000202A0ED012F5803F0BD00268546824F438
:1021A000E06454601122026380F83E1080F83D30F4
:1021B00016E00268546824F4E0645460026814680D
:1021C00044F400741460016380F83D3090F83E20C0
:1021D00080F83E10402A03D1FEF7E4FB10BD02E078
:1021E000FEF7DEFBFAE70068416821F48061416098
:1021F000F4E7BDE8104000F0F3B8000078B590F8BF
:102200003E50C26A046B90F83D6000230168222EA4
:1022100073D1066D0EB9402D6FD0056D1DB90569DE
:10222000B5F5404F1BD0458D95B3468D484D012ED9
:1022300020D0448D022C4DD00C6844F480640C6096
:1022400001684C68240579D5AA4273D0012A71D05F
:10225000082A6FD0102A6DD0202A6BD06EE04A6910
:102260008A6900920A6842F480720A60016D491C12
:10227000016578BDAA4214D10A6822F480620A601E
:1022800001684A68120504D50A6822F4806217E0E2
:10229000FFE74A698A6900920A6842F400720A609C
:1022A00050E0082A10D0202A0ED0122C0AD0042A7E
:1022B00003D0022A01D0102AE6D10A6842F48062D3
:1022C0000A603BE0012ADFD00A6822F480620A60DB
:1022D0000168DEE7042A11D0022A0FD0102A0DD09F
:1022E0000C6844F400640C6001684C698C690094CB
:1022F0000C6824F480640C6008E025E00C6844F469
:1023000080640C6001684C698969009101684C68BF
:10231000240517D5AA4207D0012A05D0082A03D0E0
:10232000102A01D0202A0DD14A6842F480524A6016
:1023300008E0FFE74A6842F480524A6001684A694F
:1023400089690091036578BD48698869009078BD06
:102350000000FFFF90F83E10402910D00169B1F550
:10236000804F19D0016DA9B3016D012910D1416CC5
:102370005FF0F10201F4407142EAD11106E0016D13
:102380000029416C05D0C9B241F00101006801612A
:10239000704701F0FE01F9E790F83D102129416CEA
:1023A00009D0C9B241F0010102681161416B29B144
:1023B000896A49B902E001F0FE01F5E7816B002965
:1023C000E6D0896A0029E3D00068416841F40061E1
:1023D00041607047FFE7416CF02201F44071CBE7A8
:1023E00010B590F83D10026D4AB1026D012A14D06B
:1023F000026D022A16D0BDE81040FFF7B1BCC16CD7
:102400000129816C02D0C1F3072108E00268C9B23A
:102410001161016D891C016510BD816CC9B2026832
:10242000116123E022291CD0428D0AB1212920D03C
:10243000428D002AF0D12129EED101684A6822F4A8
:10244000E0624A6001680A6842F400720A60002192
:102450000163202280F83D2080F83E10FEF7A2FAAA
:1024600010BD01680A6842F480720A60016D491C5F
:10247000D1E7416A026809781161416A491C4162E9
:10248000418D491E418510BD2DE9F84F0446006875
:1024900089460B9D01689846174641F480610160AA
:1024A0002068016841F48071016000954FF0011BC4
:1024B0000022594620460A9B00F080F94FF4007A2A
:1024C00040B120680068C00501D5C4F840A00320D1
:1024D000BDE8F88F216809F0FE0008612B46284905
:1024E00020460A9A00F0B2F9F0BB20684169806981
:1024F00000902A4620460A9900F03DFA40B1206C2F
:1025000004283AD12068016841F40071016034E088
:10251000FEB2B8F1010F09D02168380A08612A46D5
:1025200020460A9900F027FA0028E8D120680661C1
:102530002A4620460A9900F01EFA0028DFD12068BA
:10254000016841F4807101600095002259462046DF
:102550000A9B00F033F90028B3D1216809F0FF008D
:1025600040F00100086100E007E02B4604492046E6
:102570000A9A00F06BF90028AAD00120A8E7000011
:102580000200010038B50C4690F83D2000212825B6
:10259000954302680B4605D051699169009180F816
:1025A0003C3038BD556825F480655560E2435407DA
:1025B00000D50121120601D5828900E0028B80F846
:1025C0003C3092B2FDF7AFFF38BD00002DE9F0417D
:1025D00090F83D300446C26A002120261E4F006854
:1025E0006FF48065082A01D0202A01D1282B04D05D
:1025F000212B17D04561BDE8F081E762426822F4E3
:10260000E0624260206845612068026822F48062CE
:102610000260216384F83D6084F83E102046FEF796
:10262000BDF9E8E7E7622122226384F83D6084F87F
:102630003E10416821F4E0614160206845612068F6
:10264000016821F4806101602046FFF789FB204684
:10265000FEF71DFBCFE700000000FFFFF8B590F884
:102660003D6004460068416821F4E06141602068F3
:10267000002541690091016841F001010160206875
:10268000016821F48061016020684168090520D556
:10269000484F222E4BD02A2E49D0616B09684968D9
:1026A0006185618D19B1216C41F00401216441689B
:1026B00021F400614160606BFDF72CFE012808D019
:1026C000606B4763606BFDF7D9FD10B1606B416BC8
:1026D0008847608D20B320684169C94349070AD4FF
:1026E0000069616A0870606A00F101006062608DD3
:1026F000A0F101006085206841696FEA0101490687
:1027000008D40069616A0870606A401C6062608D6C
:10271000401E6085608D18B1206C40F0040020647C
:10272000206C00B32046BDE8F840FFF721BBA16B49
:10273000096849686185618D19B1216C41F0040116
:102740002164416821F400614160A06BFDF7E2FD66
:102750000128BED0A06B4763A06BFDF78FFD00285A
:10276000B7D0A06BB3E72A2E06D12563282084F8C2
:102770003D002046FEF78AFA94F83D1020202829D3
:102780000DD0216B222901D0222E07D1256384F898
:102790003D0084F83E502046FEF778FAF8BD064921
:1027A000E162256384F83D0084F83E502046FEF740
:1027B000F5F8F8BDA51C00080000FFFF2DE9F04763
:1027C000984617460D460446C1F30746DDF82090AB
:1027D0002AE000BF18F1010026D0FDF79DFEA0EB16
:1027E0000901414502D8B8F1000F1DD12068012E22
:1027F00016D0806925EA00000004000C12D00020E9
:10280000B84211D1002044F8300F20216173A07329
:10281000216941F02001216120730120BDE8F0878A
:102820004069E7E70120EBE72068012E0AD08069C4
:1028300025EA00000004000C06D00020B842C9D0F0
:102840000020EBE74069F3E70120F7E72DE9F047C7
:10285000984616460D4604464FF000094FF0200AF0
:10286000C1F3074723E020684069C043400515D401
:102870002068016841F40071016021686FF4806094
:102880004861C4F8309084F83DA084F83E90216CF3
:1028900041F00401216484F83C9021E0701C06D0D2
:1028A000FDF73AFEA0EB0800B04203D816B1012FA5
:1028B0001FD021E02068012F15D0806925EA000093
:1028C0000004000C18D000BF44F8309F84F80DA01D
:1028D00084F80E90216941F02001216184F80C9068
:1028E0000120BDE8F087406925EA00000004000CE3
:1028F000EAD12068406901E02068806925EA00008B
:102900000004000CAFD1ECE72DE9F0410025904622
:102910000E460446202727E04069C043C0060BD47A
:1029200054F8201B6FF01000486125616777A57788
:10293000206A2062257714E0FDF7EEFDA0EB080089
:10294000B04200D886B920684069C04340060BD524
:1029500044F8305F6773A573206940F02000206160
:1029600025730120BDE8F08120684169C94349060B
:10297000D2D40020F6E770B516460D4604461EE098
:102980002046FFF7A1FA08B1012070BD681C16D0DF
:10299000FDF7C2FD801BA84200D885B920684069B8
:1029A000C04300060BD5002044F8300F202161738E
:1029B000A073216941F0200121612073E4E72068C0
:1029C0004069C0430006DBD4002070BD0A4B0228DA
:1029D00007D021B15FF000024FF4005106E0012260
:1029E000FAE731B15FF000024FF480411846FDF77D
:1029F0008EBD0122F8E7000000100140044A0228C1
:102A000001D0511401E04FF480411046FDF777BD2D
:102A100000100140054B4FF40041012801D0012274
:102A200000E000221846FDF772BD0000000C0140D6
:102A3000044B012801D0002200E001221021184699
:102A4000FDF765BD000C014070B5104B104D4FF403
:102A50000044102806D0202806D040284FF000025D
:102A600003D108E0012206E0012208211846FDF703
:102A70004EFD002204E008211846FDF748FD012222
:102A800021462846BDE87040FDF741BD000C0140DD
:102A9000000801402DE9F04786B000243A48009430
:102AA000019402940394816941F01001816181696C
:102AB00001F010010491816941F004018161816993
:102AC00001F004010491816941F00801816180698C
:102AD000DFF8B88000F008004FF4C04504900022F1
:102AE00029464046FDF713FDDFF8A49000224AF284
:102AF0003C014846FDF70BFDDFF898A04FF4014775
:102B0000002239465046FDF702FD009503260125B7
:102B10000396CDE9015469464046FDF7FFFB009658
:102B200069465046CDE90145FDF7F8FBF020CDE9B7
:102B30000004694650460294FDF7F0FBCDE90064BD
:102B4000694648460294FDF7E9FB48F23C00CDE9AE
:102B50000005CDE9024669464846FDF7DFFB6803FC
:102B6000CDE90005CDE9025669464846FDF7D6FB9A
:102B700000970396CDE9015469465046FDF7CEFB18
:102B800006B0BDE8F08700000010024000100140D0
:102B9000000C0140000801400D4810B50B490160D0
:102BA0000C49416000214FF480428160C0E903126A
:102BB00041618161C1610162FDF732FE002803D0ED
:102BC000BDE81040FDF735BB10BD000000540040CB
:102BD000A0000020801A060010B586B00024174817
:102BE000009401940294039404944FF0804105945E
:102BF00001603F21C0E9011440F2E731C0E903144C
:102C000080218161FEF7CEFB08B1FDF712FB4FF486
:102C10008050009069460948FEF744FC08B1FDF772
:102C200008FB049404A905480594FEF787FB0028D7
:102C300001D0FDF7FEFA06B010BD0000F400002040
:102C400010B586B0002416480094019402940394B1
:102C500004941249059401603F21C0E90114322116
:102C6000C0E903148461FEF79DFB08B1FDF7E1FAAA
:102C70004FF48050009069460948FEF713FC08B1F4
:102C8000FDF7D7FA049404A905480594FEF756FB0E
:102C9000002801D0FDF7CDFA06B010BD00040040B9
:102CA0003C0100200C4810B50A4901604FF4E131A5
:102CB0004160002181600C22C160C0E90412816181
:102CC000C161FEF703FF002803D0BDE81040FDF707
:102CD000B0BA10BD00380140840100200C4810B586
:102CE0000A4901604FF4E1314160002181600C220A
:102CF000C160C0E904128161C161FEF7E7FE0028EE
:102D000003D0BDE81040FDF794BA10BD0048004064
:102D1000CC010020FEE770B505464FF6FF7000229B
:102D20004AF201040BE0AB5C58400023C6074FEAAF
:102D3000500000D060405B1C082BF7DB521C8A421D
:102D4000F1DB70BD08B50020FDF764FA0020FDF747
:102D500055FA322003460090064A07A1084800F0C1
:102D60009DF807490748C863BDE80840084600F0D9
:102D7000E0B80000CC01002055415254330000005F
:102D8000A0020020FD01000870B59AB032220DA902
:102D90003B4800F0B3F8040024D03A4D9DF83400CD
:102DA000297888421ED10DA8204430F8026CA01E5C
:102DB00081B20DA8FFF7AFFFB04213D19DF83500E7
:102DC0000C280FD006DC06280CD2DFE800F00B0739
:102DD0000D0B0B4F152805DA0F2803D121460DA83E
:102DE00000F052F81AB070BDBDF83640BDF838603A
:102DF00034216846FDF7AFF928788DF800000220ED
:102E00008DF801008DF80240200A8DF803008DF83E
:102E10000460300A8DF8050006216846FFF77BFF45
:102E20008DF80600000A8DF8070008242146684640
:102E300000F02AF82146684600F026F82146684648
:102E400000F022F82146684600F01EF82146684648
:102E500000F01AF82146684600F016F82146684648
:102E600000F012F80120FFF7C9FDBBE7BDF83800FC
:102E700020B101210120FFF7A9FDB3E70021F9E707
:102E8000A0020020300000200A460146014800F060
:102E90006AB80000A0020020FEE770472DE9F0416B
:102EA000044606986061C4E900121E4600F0ACFBBF
:102EB0004FF0FF37A06090B10025E56025612663E3
:102EC0007000A56200F0A0FB206240B13044606257
:102ED000094984F83A502564086820B908E0384662
:102EE000BDE8F0810846016C0029FBD1046400E0D4
:102EF0000C600020F4E700001C000020F0B516462E
:102F00000D46044600F052F8B04200D93046002287
:102F100013460BE02169A7684E1C2661795CA95411
:102F2000D4E90416B14200D32361521C8242F1D38A
:102F3000F0BD38B5C16B044609B1002088470120B7
:102F400084F83A0060680068016841680091C168CF
:102F500041F01001C160A08A82B2D4E90101BDE84C
:102F60003840FEF7B6BB70B504461546836A266B3B
:102F700000225819B04213D894F838002A4604EBBE
:102F80008000006A1844FDF7CDF8A06A2844A062CA
:102F900094F8390010B9204600F020F8012203E02F
:102FA000616B814200D26063104670BDD0E90312AC
:102FB0008A420FD806D1017F31B14FF0000101776D
:102FC000416901E0A1EB020182698A4200D281617C
:102FD0000846704743691944F4E7000070B5044699
:102FE000806AE16B002500B3626B824200D26063AD
:102FF00009B101208847208D82B294F8380004EB93
:103000008000016A6068FEF715FE00280AD10120E1
:1030100084F83900A56294F8380020B15FF0000010
:1030200084F8380070BD0120FAE709B10020884714
:1030300084F8395070BD704770B5234C102120467C
:10304000FDF758FA012801D0012100E000214D00D0
:1030500020212046FDF74EFA012801D0012000E092
:10306000002028434500402126462046FDF742FA2D
:10307000012801D0012100E0002129434C008021DA
:103080003046FDF737FA012801D0012000E000208A
:1030900020430E4D440001212846FDF72BFA01285C
:1030A00001D0012100E0002121434C0002212846EB
:1030B000FDF720FA012801D0012000E00020204384
:1030C00040F0400070BD000000080140000C0140CD
:1030D00038B500208DF800009DF8000040008DF804
:1030E0000000104C01212046FDF704FA012800D011
:1030F00000209DF8001008438DF800009DF80000A6
:1031000040008DF8000002212046FDF7F3F9012868
:1031100000D000209DF8001008438DF800009DF8B5
:10312000000038BD00080140704730B58FB028213D
:103130006846FDF710F814210AA8FDF70CF80225DF
:103140000120049000951020059000244FF4601099
:10315000CDE9084007956846FDF75AFF08B172B6F9
:10316000FEE70F20CDE90A054FF48060CDE90C4061
:1031700002210AA80E94FDF74FFE002801D072B676
:10318000FEE70FB030BD70470148FEF7F9B9000007
:10319000F40000200148FEF7F3B900003C010020D4
:1031A0000148FEF7EDB9000014020020F0B50268F6
:1031B000194B1A4C1A4D4FF08047984205D0B8422F
:1031C00003D0A04201D0A84203D122F070064A6881
:1031D0003243984205D0B84203D0A04201D0A84261
:1031E00003D122F44074CA6822434C6922F0800261
:1031F000224302608A68C2620A688262984201D1F0
:1032000009690163012141610169C90703D00169AD
:1032100021F001010161F0BD002C014000040040DB
:103220000008004010B5846842EA032224F47F4479
:103230000A432243826010BD826822F070020A4372
:1032400042F007018160704710B5036A046A24F0F8
:1032500001040462846924F0F00444EA021423F0B7
:103260000A020A438461026210BD10B5036A046A4F
:1032700024F010040462846923F0A00324F4704451
:1032800044EA023243EA01118261016210BD10B5C5
:10329000406A0021C185C184FEF7B4FA10BD10B5A3
:1032A000406A0021C185202280F842200163FEF798
:1032B00059FA10BD01680C3151E8002F22F49072C8
:1032C00041E80023002BF5D10168143151E8002FAB
:1032D00022F0010241E80023002BF5D1016B012906
:1032E00009D101680C3151E8002F22F0100241E8A9
:1032F0000023002BF5D1202180F84210002101632A
:10330000704708B590F84210222901D0022008BD6C
:1033100082684FF480539A4201D1016921B1816AD8
:103320009A421BD04AB10AE00268816A5268C2F32D
:1033300008020A80816A891C08E0026972B1026889
:10334000526802F07F020A70816A491C8162C18D55
:10335000491E0904090CC18503D01BE002685268AC
:10336000F1E70168CA6822F02002CA600168CA68F1
:1033700022F48072CA6001684A6922F001024A613F
:10338000202180F8421000214163026B012A03D002
:10339000FEF73CFC002008BD0163016801F10C014F
:1033A00051E8002F22F0100241E80023002BF4D155
:1033B00001680A68D20602D50A6849680091818DC1
:1033C000FEF7AEF9E6E7000010B5044600680169B3
:1033D000E26821F44051114301612169A06808436A
:1033E000616908432168CA6841F20C639A43024349
:1033F000CA6020684169A26921F4407111434161AA
:1034000013492068884202D1FDF7CCFD01E0FDF7A9
:10341000B9FD00EBC00101EB001061686422890076
:10342000B0FBF1F1B1FBF2F06FF01803434301EB95
:103430008303322101EB0311B1FBF2F101F0F00241
:1034400002EB001001F00F0108442168886010BDF4
:103450000038014081628285C285002141642221B9
:1034600080F84210016921B10168CA6842F4807293
:10347000CA6001684A6942F001024A610068C16895
:1034800041F02001C1600020704700000148FEF7B4
:10349000E5B90000840100200148FEF7DFB9000013
:1034A000CC010020FEE700000907090E002801DB1F
:1034B000034A02E0034A00F00F0081547047000005
:1034C00000E400E014ED00E002E008C8121F08C1AB
:1034D000002AFAD170477047002001E001C1121F95
:1034E000002AFBD1704700004FF08040406A02493B
:1034F00089680844704700001C000020394C08B55A
:1035000000206060FDF7CCFBFFF70FFEFFF7C2FA6B
:10351000FFF742FBFFF7C6FBFFF7E0FBFFF790FB6F
:10352000FFF75AFB3048FCF733FE304900200854BF
:10353000401C6428FBD364212C48FCF70CFE642259
:103540002A494FF48070FCF73BFEFFF775FD2070B1
:103550002078274908700020FCF75CFE0020FFF768
:1035600059FA4020FFF770FA0120FFF761FA642052
:10357000034600901F4A20A12148FFF78FFC2048F6
:10358000FFF7D7FCFFF7DEFB00F08AF81D4D2E6831
:1035900028688642FCD02E68FFF7A6FF0746FFF793
:1035A000F3FBFFF795FD6070607810B10220FFF724
:1035B00025FA64220D491248FFF7A0FCA060020022
:1035C00003D00A490E48FFF7CEFCFFF78DFFC11B61
:1035D0006068814201DB6160DAE70028D8D0401ED4
:1035E0006060D5E700000020A00000203C00002023
:1035F0003000002084010020554152543100000069
:103600005C02002028000020F0B50B30154D20F0A2
:1036100007010024144A0FE003688B420BD38B424E
:1036200005D95E1A43184768C3E9006700E043689C
:10363000136002C004E0021D10680028ECD120468F
:10364000002802D1286808B10020F0BD064A0748CA
:103650001060074A121A22F00702C0E90024012074
:103660002860D7E73800002034000020EC0200205A
:10367000E822002009484168491C4160826802F53F
:103680007A7282600522B1FBF2F302FB131100296A
:1036900002D1C168491CC160704700001C000020B5
:1036A0000148FDF7D3BE0000F40000200102020330
:1036B0000405060708090A0B0C0D0E0F1010000078
:1036C00000000000000001020304060708090000D2
:1036D0000000010203040000F8360008000000208A
:1036E0003C000000C8340008343700083C000020CB
:1036F000AC420000D83400080000000000000000C8
:1037000000000000010000001000000000000000A8
:103710000024F40000000000000000000000000091
:103720000000000000000000010000000000000098
:043730000000000095
:04000005080000ED02
:00000001FF
